:020000040000FA
:040000006D303A28FD
:08000800A000030EA100831209
:100010008B1C32288B1031181428B11C3228643004
:10002000010203183128182800001628172818285C
:1000300019281A281B281C281D281E281F283110A3
:10004000B114A810031005190314AA0DA90DA80DC9
:10005000B00B322831152A08AF002908AE00280855
:10006000AD00B11081010B11210E8300A00E200EF6
:02007000090085
:0C007400203084008001840A6030040207
:10008000031C3C281230B000A7218316FF239000E8
:10009000831283160C308505870183128501870141
:1000A000073099000030831691008312C830831600
:1000B0008100831231309000003083168C0083124F
:1000C00010308B00831600309B001C141A0883121A
:1000D000BC00851DEB21831610309B001C141A08F0
:1000E0008312BD00E32181018E018F010B118B1062
:1000F0000B108C018B178A203119A020B30B882894
:10010000031085190314B90DF030390203192221A7
:1001100010227B286400311808000B1D08000B1109
:10012000B11031141230B000051D9B283214831613
:10013000011383120800321083160117831208007E
:1001400031110130B7008B132030370783169B0025
:100150001C141A088312A400A500C030A506103094
:10016000370783169B001C141A088312A300003063
:10017000370783169B001C141A088312A2008B17E2
:10018000321CC82822090339A200A309A409A50921
:1001900022082D02031D1C2923082E02031D1C29E1
:1001A00024082F02031D1C2901303702031DDD28FE
:1001B0003D18DD283D143E14B22102303702031DE4
:1001C000E628BD18E628BD143E14B42103303702DA
:1001D000031DEF283D19EF283D153E14B6210430CC
:1001E0003702031DF828BD19F828BD153E14B821A3
:1001F00005303702031D01293D1A01293D163E1421
:10020000BA2106303702031D0A29BD1A0A29BD1674
:100210003E14BC2107303702031D13293D1B13294F
:100220003D173E14BE2108303702031D1C29BD1B9B
:100230001C29BD173E14C021B70A09303702031824
:100240000800A3280130B600B300B400B500B70021
:1002500085018701B1138A20B30B5A290310851930
:100260000314B90DF030390203198129B40B5A294E
:10027000013037020319CB21023037020319CE2196
:10028000033037020319D121043037020319D42176
:10029000053037020319D721063037020319DA2156
:1002A000073037020319DD21083037020319E02136
:1002B0009630B400311D2B293111321C64292D09CF
:1002C0000339AD00AE09AF092F1CB1132F1C2B2928
:1002D000B11B2B292E182B29B1178B132030370770
:1002E000BB002F08BA00942110303707BB002E083E
:1002F000BA00942100303707BB002D08BA009421C2
:100300008B1785018701B70AB60109303702031C34
:100310002B29E32108003E1C08003E101030BB00D2
:100320003D08BA00942108008B133A0883161C1567
:100330009A003B089B0055309D00AA309D009C14FC
:1003400064009C18A0291C1183128B170800FF3031
:10035000D000D415D515D615D715D915DA15DB1556
:10036000DC150800F130C329F230C329F430C32969
:10037000F830C3291F30C7292F30C7294F30C7296C
:100380008F30C7290800BD050F30D2040800BD0515
:10039000F030D204080010308506080020308506B1
:1003A0000800213085060800223085060800183034
:1003B00087060800213087060800093087060800F4
:1003C0002930870608003D08D200031D08001130BF
:1003D000BD00D2000800B601B301B4013C1CF329F2
:1003E000BC01BC14F529BC013C143C08B6006400F7
:1003F000F929FA29FB29FC29FD29B41B0516B41F8C
:100400000512B30BF729B40BF7290310B60CB60885
:10041000031DF7290030BB003C08BA0094210800F6
:100420008F08031908008F01D00F2A2BD00A0E3035
:100430005205031D2A2A541D202AD4015416382A95
:10044000D41D252AD4015416382A541E382AD40122
:10045000D414382AD41C2F2AD4015415382A541DF8
:10046000342AD401D415382A541E382AD4015415FC
:1004700001305205031D4B2A551D412AD501551641
:10048000592AD51D462AD5015516592A551E592ACD
:10049000D501D514592AD51C502AD5015515592AEC
:1004A000551D552AD501D515592A551E592AD5014C
:1004B00055150B305205031D6C2A561D622AD601B4
:1004C00056167A2AD61D672AD60156167A2A561E3D
:1004D0007A2AD601D6147A2AD61C712AD601561544
:1004E0007A2A561D762AD601D6157A2A561E7A2AD7
:1004F000D601561507305205031D8D2A571D832A34
:10050000D70157169B2AD71D882AD70157169B2A31
:10051000571E9B2AD701D7149B2AD71C922AD70192
:1005200057159B2A571D972AD701D7159B2A571E67
:100530009B2AD70157151030BC1811305205031DE6
:10054000B02A591DA62AD9015916BE2AD91DAB2A8F
:10055000D9015916BE2A591EBE2AD901D914BE2A5C
:10056000D91CB52AD9015915BE2A591DBA2AD90153
:10057000D915BE2A591EBE2AD90159155030BC18AA
:1005800051305205031DD32A5A1DC92ADA015A16C1
:10059000E12ADA1DCE2ADA015A16E12A5A1EE12A88
:1005A000DA01DA14E12ADA1CD82ADA015A15E12A2A
:1005B0005A1DDD2ADA01DA15E12A5A1EE12ADA018A
:1005C0005A15E030BC18E1305205031DF62A5B1DB8
:1005D000EC2ADB015B16042BDB1DF12ADB015B1629
:1005E000042B5B1E042BDB01DB14042BDB1CFB2A1E
:1005F000DB015B15042B5B1D002BDB01DB15042BE2
:100600005B1E042BDB015B152030BC18213052052A
:10061000031D192B5C1D0F2BDC015C16272BDC1D29
:10062000142BDC015C16272B5C1E272BDC01DC1451
:10063000272BDC1C1E2BDC015C15272B5C1D232BC0
:10064000DC01DC15272B5C1E272BDC015C158B21C4
:100650003D08D2005008D1000C305405031D05128E
:100660000C305505031D85120C305605031D051071
:100670000C305705031D85100C305905031D07105C
:100680000C305A05031D87120C305B05031D071241
:100690000C305C05031D871151080E020318742BE2
:1006A00012305405031D051612305505031D85161D
:1006B00012305605031D051412305705031D85140D
:1006C00012305905031D071412305A05031D8716F1
:1006D00012305B05031D071612305C05031D8715DC
:1006E000FF305002031908008F08031D08008A20FC
:1006F00051080E02031C742B18305405031D0512FB
:1007000006305405031D051618305505031D8512C6
:1007100006305505031D851618305605031D0510B6
:1007200006305605031D051418305705031D8510A6
:1007300006305705031D851418305905031D071091
:1007400006305905031D071418305A05031D87127A
:1007500006305A05031D871618305B05031D071266
:1007600006305B05031D071618305C05031D871155
:0A07700006305C05031D8715080024
:084000000400030002000600A9
:02400E00CC01E3
:10420000010003000300030003000200020002009B
:1042100002000000000000000000FF00FF00FF009F
:10422000000000000000000000000000000000008E
:104230000000C000C000C000C000FF00FF00FF0081
:104240000100C300F300CF00FF00C300F300CF0064
:10425000FF00C300F300CF00FF00FF00FF00FF00DE
:10426000FF00FF00FF00FF00FF00FF00FF00FF0056
:10427000FF00FF00FF00FF00FF00FF00FF00FF0046
:10428000FF00FF00FF00FF00FF00FF00FF00FF0036
:10429000FF00FF00FF00FF00FF00FF00FF00FF0026
:1042A000FF00FF00FF00FF00FF00FF00FF00FF0016
:1042B000FF00FF00FF00FF00FF00FF00FF00FF0006
:1042C000FF00FF00FF00FF00FF00FF00FF00FF00F6
:1042D000FF00FF00FF00FF00FF00FF00FF00FF00E6
:1042E000FF00FF00FF00FF00FF00FF00FF00FF00D6
:1042F000FF00FF00FF00FF00FF00FF00FF00AA001B
:00000001FF
